:03000000021B845C
:0C1B840078FFE4F6D8FD7581D50200362C
:0100190022C4
:06188C008B318A32893322
:101892007571027F481219F8121BD0EF20E0F9ABE4
:1018A20031AA32A9331205487879E6FE08E6FDED41
:0118B200FF36
:0118B3002212
:100F7B0043525354005341564500434647002D3EC0
:100F8B0053320052415445434C5220554E49544222
:100F9B004C4E4B545249475452455653545254534A
:100FAB00544F505A45524F44464C54534156455258
:100FBB00535420535720202E3173202E3273202E62
:100FCB00357320317320203273202035732020316C
:100FDB0030732033307320316D2020326D2020355B
:100FEB006D202031306D2033306D20316820200092
:100FFB0000000100020005000A0014003200640129
:10100B002C025804B00BB8177046508CA04665657F
:10101B0074596172644D6574724F6666204F6E2011
:10102B00204E6F2020596573204F66662054696DE2
:10103B0065416C7420547269674F66662054696D04
:10104B0065416C74204F66662054726967507772E5
:05105B00205265632036
:1018DA0025E024FAF582E4340FF583220533E53353
:1018EA00C394022208F608F608F62275F004A42426
:0518FA0024F974102226
:10142800789976AB0876CD08760008760AE408F64F
:1014380008760108F60876640876401218EE08F671
:1014480078A7F608760A08F608763C08F6087614AF
:1014580008F608760F1218EE7BFF7A0F797B1217C1
:09146800D37F0512173502183676
:101A130075751D7576C012153E789AE664CD70040F
:091A230018E664AB6003121428FC
:011A2C002297
:0D1B4C00C2AF7DC07C1DE4FF121AB6D2AFFF
:011B59002269
:10153E00753EFF85753F8576407541007542007595
:10154E004399E4FFAB3EAA3FA9408F8275830012F8
:10155E00051BAB41AA42A9438F8275830012055A1F
:10156E000FBF1AE078B2E6FFF46003EF700478B2B2
:02157E007601F4
:011580002248
:101836007D01E4FF1219837BFF7A0F79801217D39B
:10184600121B4CC2AF7F997B1A7DC07C1D121AC039
:0D185600D2AF7F02121735E4FDFF021983A7
:10097B00E4F5317BFF7A0F79851217D37F051217B8
:10098B0035A297829650FAA2969217A2979218E5E3
:10099B003175F004A4248EF9740F35F0FA7BFF1235
:1009AB0017D37F05121735853132E4F5337BFF7A88
:1009BB000F79891217D3E531B4090050779009CF1D
:1009CB00F82828730209EA020A3F020A0B020A13EB
:1009DB00020A17020A1F020A27020A2F020A377F8E
:1009EB0001EF1218DA789BE6FC08E6FD7401936DB3
:1009FB007003E4936C70028F330FBF0FE4020AC2D3
:100A0B00789DE6F533020AE8789E800278A6E6F533
:100A1B0033020B0278A5E6F533020B2978AFE6F526
:100A2B0033020B4678B0E6F533020B6378B1E6F58B
:100A3B0033020B80E5316532600302099AA217304D
:100A4B009601B35013A296921730960C0531E531EF
:100A5B00C3940C4003E4F531A218309701B350D482
:100A6B00A29792183097CDE531B40C0050C6900A7E
:100A7B0080F8282873020AA4020AD0020AD6020AB6
:100A8B00F4020B08020B1B020B34020B51020B6E10
:100A9B00020B94020B9A020BA00533E533C3940FA0
:100AAB004003753301E5331218DAE493FF740193B5
:100ABB00789BCFF608EFF6E53375F004A424BEF966
:100ACB00740F020B89121334020A3F0533E533C34B
:100ADB0094034003E4F533789DA633E53375F004B6
:100AEB00A42418F97410020B891218E64003E4F5DC
:100AFB0033789EA633E5331218F5020B891218E6EC
:100B0B004003E4F53378A6A633E5331218F5806E6F
:100B1B001218E64003E4F53378A5A633E53375F0F8
:100B2B0004A4242CF9741080550533E533C39404C5
:100B3B004003E4F53378AFA633E53375F004A42412
:100B4B0034F9741080380533E533C394034003E460
:100B5B00F53378B0A633E53375F004A42444F97467
:100B6B0010801B0533E533C394044003E4F533785D
:100B7B00B1A633E53375F004A42450F9741035F0A5
:100B8B00FA7BFF1217D3020A3F121428020A3F12F4
:0B0B9B001836020A3F43A208020A3F7E
:0A1B9C004552415300444F4E4500EE
:1019A100E4D3FCFD7B80FAF9F80206A7789BE6F503
:0D19B1005508E6F55622E56AAE6978062273
:10121500C215C216E4F532F533AE32AF331219A159
:10122500401CE53164816016AF33AE3212180512E9
:101235001AA28F310533E53370DF053280DBE531E6
:10124500B48108E533153370021532AE32AF33E49D
:10125500C31219A3700CD215121B68E4F569F56A5F
:10126500800785326985336AE4F56BF56C755480C2
:031275001219AD9E
:011278002253
:041805008F828E83BD
:101809001219A14027E582AE837806C333CE33CEC1
:10181900D8F9FD757102EE7879F6CFEDCFEF08F6BC
:0C1829007F50121A60121BD0EF20E0F973
:011835002290
:031A2D00CDEFCD2D
:101A3000757102EE7879F6ED08F67F50121A601291
:061A40001BD0EF20E0F9CD
:011A4600227D
:101AA2007571017F501219F8121BD0EF20E0F978FE
:031AB20079E6FFD3
:011AB500220E
:101A8D00121A2DE4FFFE0FBF00010EBE0FF8BFA00E
:041A9D00F5121AA282
:011AA1002222
:06176B00CBEFCBCAEECA71
:10177100301503301627757103EA7879F6EB08F610
:1017810008EDF67F50121A60121BD0EF20E0F9E449
:0D179100FFFE0FBF00010EBE0FF8BFA0F558
:01179E002228
:1015C400753400753500753654E4F5331219B7C314
:1015D40033CE33CED8F97C002533FFEC3EFEAB345A
:1015E400AA35A93685338275830012051BFD1217AF
:1015F4006B0533E533C3940640D2756B00756C06F6
:0116040022C3
:101126008E318F321219B7C333CE33CED8F9256C30
:10113600FFE56B3EFEEEC0E0EFC0E0E531FDD0E03E
:10114600FFD0E0FE12176B056CE56C7002056B12A2
:1011560019B7C333CE33CED8F9256CFFE56B3EFE07
:10116600AD3212176B056CE56C7002056B0558E520
:101176005870020557C3E56C9440E56B9400401720
:10118600E4F56BF56C056AE56A70020569AE69FF00
:081196001219A15002D215222A
:10133400E4F56BF56C7BFF7A1B799C1217D3D216FC
:10134400E4F53EF53FAE3EAF3F1219A14021E53F23
:10135400AE3E7806C333CE33CED8F9F56C8E6B7DB2
:1013640081FF12176B053FE53F70DA053E80D6C258
:10137400167BFF7A1B79A11217D3E4F569F56AF598
:051384006BF56CC215C1
:011389002241
:1012DD00E4F53EF53FF540F541AE40AF411219A1A1
:1012ED004044E53F6481603EAF41AE4012180512A7
:1012FD001AA28F3FE53F64807022AF3E053EFCFD94
:10130D00FEFBFAF9120D527F2C120016AE40AF41C2
:10131D00E4FCFDFBFAF9120D52121BB90541E54132
:06132D0070B7054080B31B
:011333002297
:021471008F3EAC
:10147300E4F53FF540F541F542AE41AF421219A103
:101483004030E5406481602AAF42AE411218051234
:101493001AA28F40E540B4800FE53F653E7007AF69
:1014A30042AE41021805053F0542E54270CB0541B6
:0214B30080C7F0
:0114B5002214
:101605001219AD78A6E6F559E4F557F5581215C443
:1016150085696D856A6E7F0112127930021A78A983
:10162500E6FE08E6FFE4FCFD7B64FAF9F812057CAA
:101635008F668E658D648C63300505C205121A7739
:011645002282
:1016FD00856931856A32E56C456B60080532E532E6
:10170D0070020531856D69856E6A1215C485316962
:10171D0085326AAE31AF321219A15007E4F569F581
:08172D006AD2157F0202127955
:101AB600740478FF769612FF0322740078FF7696F8
:041AC60012FF0322E6
:0300330002106058
:0D106000C0E0C0F0C083C082C0D075D008D1
:10106D00E5D954F8FF120720109A08109A1010A90C
:10107D001810C42010AB2810C43010C63810CC4046
:10108D0010C44810E550110258000011108574DA93
:10109D00C2DDC2DC7572007573008070800EE57163
:1010AD00700280560573E573700205721200268F6B
:1010BD00DAC2DDC2DC80558016D2DDC2DC804DC2C5
:1010CD00DDC2DCE5717004C2DA8041D2DA803DC246
:1010DD00DDD2DC756F048034AFDA121B900573E539
:1010ED007370020572C2DDC2DCE5717004C2DA8074
:1010FD001BD2DA8017AFDA121B90C2DDD2DC756F0E
:0E110D00028009756F04C2DDC2DCD2DAC2DBDB
:0B111B00D0D0D082D083D0F0D0E032E2
:1018630043910C43920CE4F5DBEF25E0F5DB3017F5
:101873000343DB0175DD2575DC2575D84453F8FE7C
:0918830053F7FEE4F56FD2E822F0
:101A6000E56F30E002FF22E4F570756F03EF25E0CB
:071A7000F574D2DD7F0222B4
:1019F800E56F30E002FF22E4F5701571756F05EFB1
:0B1A080025E04401F574D2DD7F0222CE
:061BD00020DBFDAF6F22D7
:0D0026001571AF70057074792FF8E6FF2298
:0C1B900074792570F8EFF60570157122CD
:0E1B5A00E4F5847585FFF592F5A475A5FF22CC
:071BC200EE3395E0FDFC226B
:1018FF00C212C214C211D2A2C2A0C2A1E4FDFF1231
:10190F001983E4FD7F011219837F081212797F0476
:03191F0002127938
:10198300EF146011047016BD0104C2A78002D2A730
:0E199300A2A7921322BD0103C2A622D2A62251
:10127900EF14B40800505C90128E75F003A4C58376
:1012890025F0C583730212A60212AC0212B3021230
:10129900BF0212C10212BF0212CB0212D3D21275BF
:1012A900190122C212A21392A722D214751A057D1E
:1012B900017F010219838005C211C28722C211D29E
:1012C9008722D211D28775180122C2A47F01121771
:0412D90035D2A42244
:10168500301212D5190F30A707C2A775191E80058C
:10169500D2A7751946E51AD39400400CD51A09C28C
:1016A50014E4FD7F01121983301111D5180E30870E
:0D16B50006C28775180522D28775181E22FF
:10194300C374039FFE1392A0EEA2E192A1AF80CFD6
:0F1953005480CFED547FCF4FCF8F80C2A2D2A24E
:011962002262
:0617D3008B408A418942AF
:1017D900E4FCCFECCF7D201219430CBC04F4E4FCEB
:1017E900AB40AA41A9428C8275830012051BFD609A
:0B17F9000ACFECCF1219430CBC04E532
:0118040022C1
:04119E008F828E832B
:1011A200121BC2E47B0F7A27F9F8C31206A7500379
:1011B20090270FAF82AE83121BC27B197AFC79FF94
:1011C20078FFD31206A7400390FC19E4F531741B93
:1011D2002531F8E4F60531E531B405F2AE83AF828C
:1011E200121BC27B007A00791B120D52E51E701A87
:1011F200753103741A2531F8E6FF741B2531F8C6E0
:10120200EFC6D531EE751B2080E27B007A00791B98
:031212000217D3ED
:1019BE0046554C4C0050524F47005A4C4F47004D25
:0D19CE004F440076322E35005472696700D8
:101B0600E6FE08E6FFE4FCFD2278CE1206E278C681
:031B16000206FBC9
:03001300021922AD
:10192200C0E0C0D075D010200E0CAF8DEFAD8BF59E
:101932005EEDF55FD20E758D00758B00D0D0D0E0D4
:011942003272
:021735008F3FE4
:10173700E4F540F541C3E541953FE540940050236A
:10174700900000AF82AE83E4FCFD7B207A4EF9F86F
:10175700D31206A74003A380EA0541E54170D605E9
:031767004080D2ED
:01176A00225C
:0E1B68007BFF7A1979BE1217D37F0A02173558
:0F1B3D00D20B301506121B68C20B22121605229E
:05000E00C20B0216FD0B
:101A770078D212070700000000121B0F78CE12075A
:061A870007000000002230
:10003600121B5A121BA61218FF7F0412173520979F
:10004600127BFF7A1979C31217D37F011214B6D225
:10005600AF80FE209612D2AF121A13C2177F70120B
:10006600186312121512097B7A1979C81204F7E47B
:10007600FF1214B6D2AF121A137BFF7A1979CD127A
:1000860017D378B2E62430FD7F031219437F04129A
:1000960017357A1979D11204F7C2177F70121863CF
:1000A6007F01121735121215120019C21A1216C242
:1000B6007F01121735E4F560F56112001AA29692D7
:1000C60008A2979209E4F52478CA120707000000EF
:1000D60000E4F52578D2120707FFFFD8F178C6129B
:1000E600070700000000E4F55378CE12070700006A
:1000F6000000C20DC20BC20CE4F567F568F526F5E3
:1001060027F55EF55FC20EF562C20FF55DF55CF58B
:100116005BF55AF566F565F564F563F52078AFE6A7
:1001260024FE600B14600C2402700AD2018006D2F1
:10013600068002D20078B0E624FE6007047006D27C
:10014600028002D20778B1E624FE600B14600C240C
:1001560002700AD2038006D2048002D2053001174B
:10016600C20178A7121B067B64FAF9F812057C8F88
:100176005D8E5C8D5B8C5A301AFDC21A300C33A230
:1001860008309601B3400BA209309701B340030231
:10019600026430961230970FC20CE4F567F5687F5B
:1001A60004121279E4F553A2969208A297920902D4
:1001B6000264209605209702D21030965630975347
:1001C600301031C21078C61206E2EC4D4E4F78D28E
:1001D600700C12070700000000121B0F8010120798
:1001E600070000000078C612070700000000D209C9
:1001F600D2088024789EE6601F0568E568700205CF
:1002060067D394B8E567940B400ED20C7F051212A3
:10021600798005E4F567F568A208309601B3501FAA
:10022600A2969208309618201015C201E553600771
:10023600E4F5537F0680057553017F07121279A2F4
:1002460009309701B35017A29792093097102010E2
:100256000DB20B300B05121B3D800312000E120768
:1002660046AF5DAE5CAD5BAC5AEC4D4E4F6026744E
:10027600FF2FF55DEE34FFF55CED34FFF55BEC34F6
:10028600FFF55AAF5DAE5CAD5BFC4D4E4F70062080
:100296000B03121B3DAF66AE65AD64AC63EC4D4E11
:1002A6004F602374FF2FF566EE34FFF565ED34FFDE
:1002B600F564EC34FFF563AF66AE65AD64FC4D4E98
:1002C6004F700312000E200E03020374C2AFC20E5B
:1002D600D2AFE4855F30855E2FF52EF52DAF30AEBB
:1002E6002FAD2EAC2D7B107A27F9F812057C8F30B6
:1002F6008E2F8D2E8C2DE4FB7A90F9F81214FA8F3E
:10030600308E2F8D2E8C2D78A5E66009C374B89F8C
:10031600FF740B9EFEE56214601624FE6020240323
:100326007049C3EF94B0EE9404500E7562018009D3
:10033600D3EF9414EE940540357562038030C3EF15
:1003460094B0EE94045027756201300006200B032A
:10035600121B3D300305C203121A77300B02D20F6F
:100366007BFF7A1979D61217D38003E4F562052547
:10037600E525C3940250030204F1E4F525FB7A0057
:10038600792812188C8E298F2AE5286402600302C8
:1003960004F178CA1206EEE8C0E0E9C0E0EAC0E07F
:1003A600EBC0E0789DE6FDAF2AAE291213DCD0E063
:1003B600FBD0E0FAD0E0F9D0E0F8EB2FFFEA3EFE02
:1003C600E93DFDE83CFC78CA1206FB0524E524C39A
:1003D600940550030204F178CA1206E2E47B05FA9A
:1003E600F9F81214FA78CA1206FB78CA1206E278ED
:1003F600C61206EEC3EF9BFFEE9AFEED99FDEC9852
:10040600FC78CA1206FB78D21206E278CA1206EE09
:10041600D31206A7400A78CA1206E278D21206FB61
:10042600E553600A78D4E6FE08E68E2BF52C78CCE8
:10043600E6FE08E68E29F52AE5536006AF2CAE2BBC
:100446008004AF2AAE2912119E300B4F0527E527EF
:1004560070020526C3789C96E5261896403DE4F57D
:1004660026F5277F03121279300D0DE529FF1200BC
:1004760016AF2AE52A12001620151A78A6E6600C91
:10048600300F097F007E82121126C20FAF2AAE29D5
:100496001211268006121B6812000E78CA1206E296
:1004A60078CE1206FB78CA12070700000000E4F5B2
:1004B60024300405C204121A7730061678AB121BD4
:1004C6000678CE1206EED31206A74006200B0312BC
:1004D6001B3D30071678AD121B0678CE1206EEC30A
:1004E6001206A75006300B0312000E1216850201E3
:0104F6007D88
:0B04F7007BFF1217D37F041217352281
:1018B400444C0021536967005A4C4F47004D4F4434
:1018C40000322E35004175672033312032303034F8
:0618D4000050524F4700D6
:10158100AF39AE38AD37AC36EC4D4E4F22EF24FFBC
:10159100F539EE34FFF538ED34FFF537EC34FFF56E
:1015A1003622E475392075384EF537F53622E47563
:1015B1003901F538F537F536227533007534007584
:0315C10035992237
:10074600121B76EF700302095B7F04121279E4F53F
:1007560053C20CF567F5681219DBEF120720093F43
:100766002409482A094B50089852078C61081A63D5
:10077600086D6C087372087073089C74090F76090B
:1007860007780000095B7BFF7A1879B41217D31239
:1007960015A3121B76EF700A121581600512158ECD
:1007A60080F0121581700302095B1219DB8F321279
:1007B6001471E4F5391215B3E47F06FEFDFCAB397E
:1007C600AA38A937A836C31206BD501F121AA28F1F
:1007D60032120016E5392401F539E43538F538E4E6
:1007E6003537F537E43536F53680CD121AA28F3215
:1007F600E53264806016E5326481601012001612DC
:100806001AA28F321200167531018003E4F531E524
:100816003170D8221215BA1215AFF5321215816051
:10082600241215A3121B76EF700A121581600512A9
:10083600158E80F0121581600312095C0532E532CF
:10084600C3941A40D7121581601A7899B6AB070877
:10085600B6CD030209457BFF7A1879B71217D37F05
:100866000A021735020904B20D220212DD1215BA68
:10087600E4F532AB330535E535AA34700205341498
:10088600F9120502FF1200160532E532C3941A402A
:10089600E22243A2082275330075340075357712BB
:1008A60015AFF53212158160241215A3121B76EFCF
:1008B600700A121581600512158E80F0121581607E
:1008C6000312095C0532E532C3940240D712158142
:1008D600602CAE77AF78EE3395E0FDFC78CE12064D
:1008E600EEC3EF9BF53DEE9AF53CED99F53BEC98A2
:1008F600F53AAF3D78A3E53CF608EFF680410215E0
:100906003E7F041212790213347A1879BC120970E8
:100916007A1879C1121B1978B2E62430FF12001634
:10092600121BB97F761200167A1879C51209707AE9
:100936001879C9121B19021BB9E478A3F608F60246
:1009460018360214287BFF7A1879D51217D37F013F
:050956001214B680FE42
:10095B00221219DBAB33AA34A93585328275830099
:10096B00EF12055A227BFF121B19121BB97BFF22B8
:0A1BA600E4F5955396BF53A27F2289
:1016C2005389F0438901538FFE758C70E4F58A5378
:1016D200B8FD53B7FDD2A9D28C53890F43899053D9
:1016E2008FEFF58DF58B4391105392EF53B8F7536B
:0B16F200B7F7D2ABD28ED28AD2AA2268
:03000B00021BB025
:091BB000D21A758C70758A00329E
:03001B00021BC9FC
:071BC900758D00758B0032E1
:101ACA000D0A003031323334353637383941424322
:041ADA004445460039
:101ADE00AF52AB46AA47A948055222AF45AE44AD18
:041AEE0043AC4222A1
:1014B6005387BF75985053877FE4F5BABF0105433C
:1014C600A240800353A2BFE4F5BD75BE30F5BF75DB
:1014D600BD035391FE4392014391025392FDC21BF9
:1014E60053B8EF53B7EF43B81078C4F618F678C57B
:0414F600F6D2AC225C
:0300230002179F22
:10179F00C0E0C0D075D01030981E78C4E6C3940F47
:1017AF00501418E60624B3F8A69978C40618E6C3B1
:1017BF00941040027600C298309904C299C21BD08F
:0417CF00D0D0E03264
:08000300201BFDD21B8F992286
:1019630078C4E6D39400401508E60624B3F8E6FFEE
:0F19730078C41608E6C394104005E4F6227F00FE
:011982002242
:03001600020003E2
:1019DB007F207E4E78C4E67010D3EF9400EE940017
:0C19EB004007EF1F70EE1E80EB12196326
:0119F70022CD
:101B1900120502FF600C120016740129F9E43AFA61
:031B290080EE2229
:0E1B760078C4E6D3940040037F01227F002252
:101A4700CEEFCEEE54F0C4540F901ACD93FF120090
:091A570016EE540F93FF02001675
:101B2C00CDEFCDCCEECCEEFF121A47CFEDCF021A93
:011B3C004761
:091BB9007BFF7A1A79CA021B199C
:0E0D52008F458E448D438C428B468A478948DC
:100D6000E4F552EC4D4E4F7017E94A4B70057F3059
:100D7000020016121ADE8F827583007430020E751F
:100D8000121AEBEC33502AE5484547454670077F79
:100D90002D120016800D121ADE8F82758300742DBD
:100DA00012055A121AE91206998F458E448D438C0A
:100DB00042755101754C00754BCA754A9A75493B8D
:100DC000E4FFFEFDFCAB4CAA4BA94AA849D312068E
:100DD000BD5003020E60121AE9A8491206078F508F
:100DE0008E4F8D4E8C4DEC4D4E4F7004E55170235F
:100DF000E5502430FFE5484547454670051200168A
:100E0000800EAE52121AE08E82758300EF12055AE0
:100E1000E4F551AF4CAE4BAD4AAC49AB50AA4FA92B
:100E20004EA84D12057CC8ECC8C9EDC9CAEECAC3AC
:100E3000E5459FF545E5449AF544E54399F543E5D5
:100E40004298F542AF4CAE4BAD4AAC49E47B0AFA4E
:100E5000F9F81206078F4C8E4B8D4A8C49020DC053
:100E6000E547454845466010AB46AA47A948855224
:080E700082758300E412055AAB
:010E78002257
:100BA6000134C35001DBBF68028BBB800344B79896
:100BB6000407B3B004D5AFC805A9ABE00689A7F80A
:100BC6000775A410086DA02809719C400A819858E1
:100BD6000B9F94700CCA90880DE98CF90E048CA0BA
:100BE6000EA88AAC0F4D88B80FF786C410A184D022
:100BF600115182DC120580E812BB7EF413747D006D
:100C060014307B0C14F2791815B8772416807530D9
:100C1600174B733C1819714818ED6F5419C46D6061
:100C26001AA16B6C1B7E69781C6167841D4A6590EE
:100C36001E37639C1F2561A8201A5FB421125DC070
:100C4600220D5BCC230E59D8241557E4251F55F0E9
:100C5600262F53FC27425208285B501429764E2033
:100C66002A9B4C2C2BC04A382CEE48442E1E46504C
:100C76002F55445C308F426831D1407433173E8023
:100C860034633C8C35B13A98370938A4386636B0A7
:100C960039C734BC3B2D32C83C9D30D43E0F2EE0C4
:100CA6003F882CEC41062AF8428D29044418271067
:100CB60045AB251C4741232848E121344A861F407D
:100CC6004C311D4C4DE21B584F9C1964515D1770F9
:100CD6005323157C54EF138856C4119458A20FA0C1
:100CE6005A830DAC5C6D0BB85E6009C4605807D0C2
:100CF600625A05DC646203E8667301F4688A0000E0
:100D06006AA1FE0C6CB8FC186ECFFA2470E6F830B7
:100D160000000000000000000000000000000000CD
:100D260000000000000000000000000000000000BD
:100D360000000000000000000000000000000000AD
:0C0D4600000000000000000000000000A1
:1016460075F004E538A424A6F582E5F0340BF5839D
:10165600E49322FE740193FF75F004E538A422F5A5
:1016660083C37401939FFFE4939EFEE4228F398E19
:0F167600388D378C36228F358E348D338C32225F
:101AF200C3EF9DEE9C400AD3EF9BEE9A50037F0109
:041B0200227F00221C
:040E79008E368F37EB
:100E7D00E4F538121646FC740193FD12165E24AA91
:100E8D00F582E5F0340BF583E493FA740193FBAF2F
:100E9D0037AE36121AF2EF7003020F6912164612B0
:100EAD00165924AAF582E5F0340B1216658F3C8E87
:100EBD003BF53AF53912165E24ACF582E5F0340BAC
:100ECD00F583E49312165924A8F582E5F0340B123C
:100EDD0016658F408E3FF53EF53DAD3EAC3D12069D
:100EED00998F408E3F8D3E8C3DAE36AF37E4FCFD85
:100EFD00EEC0E0EFC0E0121646FE740193FBCAEEA1
:100F0D00CAD0E0FFD0E0FEC3EF9BFFEE9AFEED945A
:100F1D0000FDEC9400FCAB40AA3FA93EA83D120594
:100F2D007CAB3CAA3BA93AA8391214FAC8ECC8C943
:100F3D00EDC9CAEECACBEFCB12165E24A8F582E539
:100F4D00F0340BF583E493FE740193FFE4FCFDEBA9
:100F5D002FFFEA3EFEED39FDEC38FC220538E53871
:0D0F6D00C3946A5003020E80E4FFFEFDFCF9
:010F7A002254
:01001A0022C3
:10138A00121673AB39AA38A937A836E8C0E078A193
:10139A00E6FE08E6FFE4FCFDD0E0F812057C121632
:1013AA0073780E1206CE12167378A3E6FE08E6FFCD
:1013BA00EE3395E0FDFCE5392FF539E5383EF53891
:1013CA00E5373DF537E5363CF536AF39AE38AD375A
:0213DA00FC22F3
:0213DC008D3151
:1013DE00120E7912167C12138A12167CE5311460E5
:1013EE001C14702DE47FE87E03FDFCAB35AA34A9F6
:1013FE0033A83212057CE47BE87A0B800CAF35AE55
:10140E0034AD33AC32E47B03FAF9F81214FA121647
:09141E007CAF35AE34AD33AC32C5
:0114270022A2
:10050200BB010689828A83E0225002E722BBFE02F7
:09051200E32289828A83E493222A
:10051B00BB010CE58229F582E5833AF583E0225095
:10052B0006E92582F8E622BBFE06E92582F8E222DF
:0D053B00E58229F582E5833AF583E49322F9
:10054800BB010689828A83F0225002F722BBFE0192
:02055800F3228C
:10055A00F8BB010DE58229F582E5833AF583E8F0D7
:10056A00225006E92582C8F622BBFE05E92582C883
:02057A00F2226B
:10057C00E88FF0A4CC8BF0A42CFCE98EF0A42CFC1E
:10058C008AF0EDA42CFCEA8EF0A4CDA8F08BF0A49C
:10059C002DCC3825F0FDE98FF0A42CCD35F0FCEBFB
:1005AC008EF0A4FEA9F0EB8FF0A4CFC5F02ECD39C0
:0F05BC00FEE43CFCEAA42DCE35F0FDE43CFC222D
:1005CB0075F008758200EF2FFFEE33FECD33CDCCE7
:1005DB0033CCC58233C5829BED9AEC99E58298406A
:1005EB000CF582EE9BFEED9AFDEC99FC0FD5F0D647
:1005FB00E4CEFBE4CDFAE4CCF9A88222B800C1B971
:10060B000059BA002DEC8BF084CFCECDFCE5F0CBAE
:10061B00F97818EF2FFFEE33FEED33FDEC33FCEBE7
:10062B0033FB10D703994004EB99FB0FD8E5E4F9A2
:10063B00FA227818EF2FFFEE33FEED33FDEC33FC8F
:10064B00C933C910D7059BE99A4007EC9BFCE99A83
:10065B00F90FD8E0E4C9FAE4CCFB2275F010EF2FC8
:10066B00FFEE33FEED33FDCC33CCC833C810D707C8
:10067B009BEC9AE899400AED9BFDEC9AFCE899F803
:0E068B000FD5F0DAE4CDFBE4CCFAE4C8F92296
:1014FA00C2D5E830E70FB2D5E4C39BFBE49AFAE41D
:10150A0099F9E498F8EC30E717B2D51215301206BB
:10151A0007E4C39BFBE49AFAE499F9E498F8800398
:10152A0012060730D50DE4C39FFFE49EFEE49DFD3D
:04153A00E49CFC220F
:0E069900C3E49FFFE49EFEE49DFDE49CFC2272
:1006A700EB9FF5F0EA9E42F0E99D42F0EC6480C8CA
:0606B70064809845F0226A
:1006BD00EB9FF5F0EA9E42F0E99D42F0E89C45F093
:0106CD00220A
:1006CE00E86010ECA2E713FCED13FDEE13FEEF1342
:0406DE00FFD8F0222F
:0C06E200E6FC08E6FD08E6FE08E6FF2244
:0D06EE00E6FB08E6F908E6FA08E6CBF8227C
:0C06FB00ECF608EDF608EEF608EFF6222B
:10070700D083D082E493F608740193F608740293B9
:09071700F608740393F6740473F0
:10072000D083D082F8E4937012740193700DA3A368
:1007300093F8740193F5828883E47374029368607C
:06074000EFA3A3A380DF7C
:00000001FF
